:100000000C9438000C9453000C9453000C9453003F
:100010000C947E040C9453000C9453000C945300E5
:100020000C9453000C94E3030C9453000C94530071
:100030000C9453000C9453000C9453000C945300F4
:100040000C940F040C9453000C9453000C943F0731
:100050000C94280E0C9453000C9453000C945300F1
:100060000C9453000C9453000C9453000C945300C4
:1000700011241FBECFEFD4E0DEBFCDBF12E0A0E061
:10008000B1E0E0EDF8E302C005900D92A038B107B1
:10009000D9F714E0A0E8B2E001C01D92A230B10788
:1000A000E1F70C940F060C9400009091AC02292FFC
:1000B000221F2227221F892F82958695869583707D
:1000C0002827892F82958F702827892F86958695D6
:1000D00028272170892F9927880F991F282B209373
:1000E000AC02822F99270895FF920F931F93F894E3
:1000F000809182028150823000F180918D028630A1
:1001000010F010928D0280918D0280FF02C09498B1
:1001100004C0949A88EF0E94230880918D0288235E
:1001200039F080918D028F5F80938D02789447C360
:1001300080918D028F5F80938D028091810280FF7C
:10014000E4C18091D70299278830910541F1893027
:10015000910594F48330910509F48AC084309105A7
:100160001CF4019721F10AC38530910509F41EC1E1
:10017000079709F4A1C002C38B30910509F49CC014
:100180008C30910524F4099709F410C1F7C28D3021
:10019000910509F40BC10F9709F48EC0EFC280E0FE
:1001A0000E94660F8091A7020E94F108E7C2809129
:1001B0008D03882321F480918203882361F090913C
:1001C000A7029F3F41F0991F9927991F8091A30291
:1001D000892B0E94660F80918203882309F4CEC286
:1001E00080918A03803150F480918A03E82FFF27A1
:1001F000E057FC4F80818F3F09F0C0C210928A0304
:10020000809189038F5F8093890380918903803176
:1002100068F480918903E82FFF27EE0FFF1FEE5946
:10022000FC4F808191818F5F9F4F11F41092890361
:1002300080918903E82FFF27EE0FFF1FEE59FC4F37
:1002400080819181909385038093840380918403BE
:10025000909185038F5F9F4F21F48FEF80939003E0
:100260008DC20E94F21080939D020E94F40B86C200
:1002700080918D03882309F481C28091A7028F3F6A
:1002800029F0881F8827881F0E94660F80918A03A3
:100290008F5F80938A0380918A03803150F480912C
:1002A0008A03E82FFF27E057FC4F80818F3F09F03A
:1002B00065C210928A0362C28091E103882309F427
:1002C0005DC29091A7029F3F41F0991F9927991F06
:1002D0008091A302892B0E94660F2091A702822F92
:1002E00099278F739070892B21F080919D02820F46
:1002F00001C0822F0E94F10880918A03803150F45E
:1003000080918A03E82FFF27E057FC4F80818F3FC1
:1003100009F034C210928A038091E0038F5F8093CA
:10032000E0038091E003803248F48091E003E82FFD
:10033000FF27E054FC4F80818F3F11F41092E003BF
:1003400060EC73E080EA93E00E94B318882331F0F8
:100350009091A1028091A0029817A1F0A0EAB3E0C9
:10036000E0ECF3E09FE18D918193915097FFFBCFFB
:100370001092E00310929D0210929C020E94FF0CCA
:100380000E94A80D8091A0028093A10280919C02FE
:1003900080939D028091E003E82FFF27E054FC4FFB
:1003A00060818091A1020E943915E8C18091E1032A
:1003B000882309F4E3C19091A7029F3F41F0991F60
:1003C0009927991F8091A302892B0E94660F209183
:1003D000A702822F99278F739070892B59F0109163
:1003E0009D02120F80918403909185030E94DD107D
:1003F000810F01C0822F0E94F10880918A03803111
:1004000050F480918A03E82FFF27E057FC4F80814A
:100410008F3F09F0B3C110928A0380918903803124
:1004200070F480918903E82FFF27EE0FFF1FEE592C
:10043000FC4F808191818F5F9F4F09F050C01092D7
:1004400089038091E0038F5F8093E0038091E00354
:10045000803248F48091E003E82FFF27E054FC4FFE
:1004600080818F3F59F51092E00360EC73E080EAE1
:1004700093E00E94B318882331F09091A1028091FB
:10048000A002981791F0A0EAB3E0E0ECF3E09FE15E
:100490008D918193915097FFFBCF10929D02109206
:1004A0009C020E94FF0C0E94A80D8091A0028093E4
:1004B000A10280919C0280939D0205C08091E0037F
:1004C0008F5F8093E0038091E003E82FFF27E054E3
:1004D000FC4F60818091A1020E947E1105C0809135
:1004E00089038F5F8093890380918903E82FFF2719
:1004F000EE0FFF1FEE59FC4F808191819093850391
:10050000809384030E94F21039C18091D702992709
:100510008830910541F18930910594F4833091053B
:1005200009F48EC0843091051CF4019771F126C145
:100530008530910509F4BFC0079709F4B2C01EC108
:100540008B30910509F4ADC08C30910524F40997E6
:1005500009F4B1C013C18D30910509F4ACC00F97F7
:1005600009F49FC00BC18091A70280938002809103
:10057000A6028093A7020E9455008093A602809154
:10058000A70240E0642F8F73F3C080918D0388230E
:1005900029F480918203882309F4F0C080918D03AF
:1005A000882379F080918A03803148F480918A030E
:1005B000E82FFF27E057FC4F80818F3F11F4109206
:1005C0008A036091A7026093800280918A03E82FDA
:1005D000FF27E057FC4F8F5F80938A03E081E09311
:1005E000A702EF3F09F4CAC08091A202882319F044
:1005F000E07CE093A7022091A702822F99278F73B6
:100600009070422F4295469546954370661F662727
:10061000661F2F73892B59F041708091A402482BDB
:100620008091A302682B80919D02820F37C0417098
:100630008091A402482B8091A302682B822F2EC0A8
:1006400080918D03882309F499C00E94F40B809156
:100650008A030E94060C8091A702809380028091F9
:100660008A03E82FFF27E057FC4F80818093A70281
:100670008F3F09F483C00E943F0D2091A702922F63
:100680009295969596959370917080918002881FAF
:100690008827881F492F682F822F8F730E944B0F46
:1006A0006DC08091E103882331F00E94F40B8091AA
:1006B0008A030E94060C8091E103882309F45EC03E
:1006C0000091A7020093800280918A03E82FFF2700
:1006D000E057FC4F8F5F80938A03E081E093A7028D
:1006E000EF3F09F44BC08091A202882319F0E07C0F
:1006F000E093A7022091A702822F99278F73907011
:10070000422F4295469546954370602F661F662797
:10071000661F2F73892B21F151E0F52EF422809171
:10072000A402F82A0091A302062B10919D02120F39
:1007300080918403909185030E94DD104F2D602FDE
:10074000810F0E944B0F1091A70280919D02180FFC
:1007500080918403909185030E94DD10810F0CC06D
:1007600041708091A402482B8091A302682B822FB4
:100770000E944B0F8091A7020E94CD0880918102B8
:10078000843030F485E20E94510B0E949A0D09C01A
:1007900080918102883028F485E20E94B30B0E9488
:1007A0008D0D0E947C0D809181028F5F809381026C
:1007B00080918102883010F01092810278941F910C
:1007C0000F91FF9008951F920F920FB60F92112470
:1007D0002F933F934F935F936F937F938F939F9349
:1007E000AF93BF93EF93FF938091AD029091AE02D0
:1007F00090938900809388000E947400FF91EF918C
:10080000BF91AF919F918F917F916F915F914F9128
:100810003F912F910F900FBE0F901F9018951F9230
:100820000F920FB60F9211242F933F934F935F9324
:100830006F937F938F939F93AF93BF93CF93EF93D8
:10084000FF9380918E028F3F29F080918E028F5FFF
:1008500080938E0280919E0290919F028F5F9F4FA6
:1008600049F080919E0290919F02019690939F0281
:1008700080939E0280918B0290918C02892B81F053
:1008800080918B0290918C02019790938C028093BF
:100890008B0280918B0290918C02892B09F49498A1
:1008A000809182028130C1F4C0B3C295CF70C17013
:1008B00080918802882371F4CC2361F080918C02AE
:1008C00090918D02019690938D0280938C0288EF17
:1008D0000E942308C0938802FF91EF91CF91BF91AE
:1008E000AF919F918F917F916F915F914F913F91C8
:1008F0002F910F900FBE0F901F9018951F920F927F
:100900000FB60F9211242F933F938F939F9329B388
:1009100023708091AF02281791F1833041F4223087
:1009200099F48091AA029091AB02019709C082309C
:1009300059F4233049F48091AA029091AB020196B8
:100940009093AB028093AA028091AA029091AB028D
:100950008D52914030F08CE291E09093AB02809305
:10096000AA028091AA029091AB02449730F484E1EC
:1009700090E09093AB028093AA022093AF029F91E4
:100980008F913F912F910F900FBE0F901F90189550
:1009900043E350E081B1886981B940B920E030E09B
:1009A0002CBF4FE150E08AB188698AB949B920BDAE
:1009B00080EC8ABB8CE38BBB8BEB87BB18BA8FEFC9
:1009C00084BB81BB86B981E58DB9089589B7816003
:1009D00089BF8BE083BF8AEF81BF089580917D003E
:1009E000846080937D00089585E20E94B30B80911E
:1009F0007D008B7F80937D000895E199FECF9FBBA2
:100A00008EBBE09A8DB39927089580917D008695DD
:100A100086959927817090700895E199FECF9FBBCC
:100A20008EBB6DBBF894E29AE19A789408950F9387
:100A30001F93CF93DF938C0181E00D32180710F0E4
:100A40000CE211E00431110510F404E110E0109300
:100A5000A9020093A8021093AB020093AA02812F6F
:100A60009927682F85E090E00E940D056091A8020B
:100A700086E090E00E940D058091A8029091A90265
:100A80000E94E90DC0E0D0E7E8E3F9E398014427CC
:100A90005527BE01CF010E94461CFA01E90193E0EF
:100AA000F695E795D795C7959A95D1F7BE01CF01F1
:100AB00026E030E040E050E00E94461CFA01E901E7
:100AC000CA01AA27BB279C01009731F4D093AE023C
:100AD000C093AD0281E061C0887F892B69F403E097
:100AE000F695E795D795C7950A95D1F7D093AE02BD
:100AF000C093AD0282E051C0C901807F892B69F4A7
:100B000014E0F695E795D795C7951A95D1F7D09348
:100B1000AE02C093AD0286E040C0C901807E892B41
:100B200069F4B5E0F695E795D795C795BA95D1F7ED
:100B3000D093AE02C093AD0287E02FC0C901807C84
:100B4000892B69F4A6E0F695E795D795C795AA9500
:100B5000D1F7D093AE02C093AD0283E01EC0C901AD
:100B60008070892B51F48D2F9E2FAF2FBB27909330
:100B7000AE028093AD0284E010C020703C7F232B36
:100B800079F46AE0F695E795D795C7956A95D1F718
:100B9000D093AE02C093AD0285E080938A0002C07C
:100BA00010928A008091AD029091AE02909581954D
:100BB0009F4F9093AE028093AD02909389008093F3
:100BC0008800DF91CF911F910F9108950F931F938C
:100BD00080916B00816080936B0080916B008260DC
:100BE00080936B008BB788608BBF85E090E00E949C
:100BF000FD049927182F002786E090E00E94FD044D
:100C00009927802B912B0E941705109281028091C9
:100C10007D00846080937D001F910F910895CFEF38
:100C2000D4E0DEBFCDBF0E94C8040E94E6050E944A
:100C3000E6048091A8028093AC020E946B090E9496
:100C4000910778940E94B7098091D702992788303C
:100C5000910509F453C089309105CCF48330910596
:100C600071F18430910554F48130910569F182303D
:100C700091050CF052C0892BB9F1E4CF8530910574
:100C800059F185309105ACF1079731F1DBCF8C300C
:100C9000910509F442C08D3091051CF40A97E9F1E1
:100CA0001DC08E30910531F08E30910594F00F9774
:100CB00081F0C8CF109282020E94400FC3CF1092E1
:100CC00082020E94E215BECF109282020E94EB11B6
:100CD000B9CF1092820205C081E001C082E080930A
:100CE00082020E94CC18AECF109282020E94350878
:100CF000A9CF109282020E946D0FA4CF109282029F
:100D00000E94EE040E94DF0B0E94B7098091D70277
:100D10008830D1F30E94F40495CF0E94DF0B0E942B
:100D20007C0D90CF159BFECF83B980E090E00895B5
:100D3000CF93DF93EC018881882331F089910E9461
:100D4000920688818823D1F7DF91CF9108950F9380
:100D50001F93CF93DF93EC0100E117E2CE01B801BE
:100D60000E94321C6115710581F0862F805D0E9402
:100D70009206CE01B8010E94321CEC01C8016AE063
:100D800070E00E94321C8B010EC0CE01B8010E949F
:100D9000321CEC01C8016AE070E00E94321C8B0139
:100DA0006A307105D8F601151105A9F0CE01B80118
:100DB0000E94321CCB01805D0E949206CE01B801D8
:100DC0000E94321CEC01C8016AE070E00E94321CF3
:100DD0008B01672B59F7DF91CF911F910F910895E8
:100DE0008F708A3010F4805D01C0895C0E94920689
:100DF00008950895CF93DF93EC01892F9927829569
:100E00008F70009711F00E94F0068D2F99270097A0
:100E100011F00E94F006CE0144E0969587954A9520
:100E2000E1F7009711F00E94F0068C2F0E94F00667
:100E3000DF91CF91089582B1992787FD90958827FA
:100E4000990F881F99270895179BFECF83B1992783
:100E5000089520EA3FE0E22FF32F3197F1F78A95CA
:100E6000D1F708958AEF0E9429078AEF0E94290787
:100E70008AEF0E9429078AEF0E94290708951F928E
:100E80000F920FB60F9211248F939F93EF93FF93BE
:100E90009CB1983FB1F480918202813021F0949A04
:100EA00085E080938B028091E103882349F1809152
:100EB000830290918402019690938402809383022E
:100EC0001FC080918602E82FFF27EF54FD4F9083CB
:100ED0008F5F80938602809186028F718093860255
:100EE0009091860280918702981751F48091870231
:100EF0008F5F80938702809187028F718093870232
:100F0000FF91EF919F918F910F900FBE0F901F90C7
:100F1000189599270E94FD04803108F08FE09927E9
:100F2000089583E00E9489078093D10284E00E94A3
:100F300089078093B002089590918702809186027C
:100F4000981719F081E090E0089580E090E008950E
:100F5000089590918702809186029817D1F3F894B2
:100F600080918702E82FFF27EF54FD4F8F5F80931A
:100F700087029081809187028F7180938702789495
:100F8000892F992708950E949C07892BC1F00E9400
:100F9000A90787FF14C0682F62956F70482F5527E7
:100FA0006F3059F09A012F7030708091D1029927DB
:100FB0002817390721F460938502CA01089580E05B
:100FC00090E00895089590918002891741F480E09F
:100FD0000E94660F0E94110D8FEF8093800208958A
:100FE0000895FF920F931F93CF93C82F00E0F02E28
:100FF000662321F4602F0E94E30720C080918002C5
:101000008F3F09F001E0653610F081E0F82E1C2FCB
:1010100019514F2D602F812F0E944B0F812F0E945D
:101020003F0D81E0F81619F48F2D0E94510B01300D
:1010300019F482E00E94510BC0938002CF911F915E
:101040000F91FF9008955D9BFECF8CB980E090E0FA
:1010500008958091B002806B0E9423088BE70E9464
:10106000230880E00E94230808951F93CF930E94D5
:10107000F4040E94F40B8091D1020E94060C10919E
:10108000DE028FEF809380020E94B7098091D70221
:10109000882319F00E9429087DC00E944B0B8823E9
:1010A00039F1412F55278091DE02992701969C0145
:1010B000207F3170821B930B2091D1024817590772
:1010C00021F4222339F0215003C02F3019F02F5F73
:1010D0002093D1026091D10283E090E00E940D053F
:1010E0000E94F40B8091D1020E94060C1091DE0246
:1010F0000E949C07892B41F20E94A907C82F482F04
:10110000441F4427441F89F0582F52955F705F3069
:1011100051F099278F7090702091D1023327821758
:10112000930709F0B1CF50938502809185029927EA
:101130008930910551F08A3091051CF4089789F0A7
:101140001CC00E9709F4A0CF18C0442319F00E94C8
:10115000A907C82F0E94A907682F8C2F0E94F107AA
:1011600093CF442319F00E94A907C82F0E94A90712
:10117000682F8C2F0E94E30787CF83E091E00E94C5
:1011800098068C2F99270E94FA068DE191E00E9423
:1011900098067ACFCF911F910895CF93C82F809151
:1011A000B00280690E9423088C2F99278F7390705A
:1011B000892B11F480E003C08C2F8F73875E0E940F
:1011C00023088C2F829586958695837080FF03C0B7
:1011D0008091020102C0809100010E942308CF91FA
:1011E0000895CF93C82F8091B00280680E94230891
:1011F0008C2F99278F739070892B11F480E003C096
:10120000CF738C2F875E0E942308809101010E947A
:101210002308CF91089580918202823029F08CEFCB
:101220000E9423080E94290808950895CF930E94E0
:101230000505C82F809182028130D1F0CC2311F0B6
:101240000E94F4049498979A85E00E94290780915F
:10125000AD029091AE020A97909389008093880026
:1012600010928D0210928102CC2311F00E94EE04A4
:10127000CF91089580918202813009F09798089566
:10128000089590B3991F9927991F80918A02882306
:1012900039F4992329F090938A0281E090E008952F
:1012A00090938A0280E090E00895089590B3991F8A
:1012B0009927991F80918902882339F0992329F46D
:1012C0009093890281E090E008959093890280E0F4
:1012D00090E00895089581B3806F81BB82B38F70D1
:1012E00082BB08958FE091B3982391BB92B398236A
:1012F00092BB0895DE980895AC01F894C098000060
:10130000000000000000C09A20E01FB8779BFECFCD
:10131000FA01E20FF11D8FB180832F5F2330A8F314
:101320007894089599B3969596959F70292F269550
:1013300026952695892F86958270282B892F9927A7
:10134000880F991F382F3470232B880F991F880F0F
:10135000991F8870282B8FE0821B99270895DE9AA9
:10136000089589B3869586958F7099270895AF92D1
:10137000BF92CF92DF92EF92FF920F931F93CF9382
:10138000DF93CDB7DEB726970FB6F894DEBF0FBE5A
:10139000CDBF2091AA023091AB028091A80290911A
:1013A000A9022817390731F08091AA029091AB0267
:1013B0000E941705ABEDB2E0E4EDF2E042E01192DD
:1013C0001D92415047FFFBCF80918E02843108F47B
:1013D00090C010928E020E947A09CE0101960E945E
:1013E0007C098091D8028C838091D9028D83809171
:1013F000DA028E8340E001E010E05E01A00EB11E33
:10140000842F869586958695A82FBB27BD016852A7
:101410007D4F842F8770980102C0220F331F8A9559
:10142000E2F7C901FB013081232F2823FD01E1529E
:10143000FD4FE081E823AA0DBB1DAC91A8234F5FAF
:101440008095222319F03823EA2B02C03823EA239F
:101450003E2BFB013083483198F20E949209482FBD
:101460008091DE02481749F08091D302481729F491
:101470004093DE0281E080938F024093D3020E946A
:10148000AF096BEDC62E62E0D62E54EDE52E52E08C
:10149000F52E08ED12E0BE016C5F7F4FAFEDB2E0BC
:1014A00042E0F50181915F018D93FB012191BF0124
:1014B000F80181918F01922F98278923F701819359
:1014C0007F019223F60191936F01415047FFE9CFCD
:1014D0000E94B109482F8091D702481731F08091BE
:1014E000D202481711F44093D7024093D2020E94CF
:1014F0007C0D26960FB6F894DEBF0FBECDBFDF91F0
:10150000CF911F910F91FF90EF90DF90CF90BF9000
:10151000AF900895282F883118F080E090E008956A
:10152000869586958695E82FFF27E852FD4F8081A6
:101530009927277002C0959587952A95E2F79C0117
:101540002170307080FF03C081E090E00895C901F0
:1015500008950895282F883118F080E090E00895CC
:10156000869586958695E82FFF27EC52FD4F808162
:101570009927277002C0959587952A95E2F79C01D7
:101580002170307080FF03C081E090E00895C901B0
:1015900008950895282F883118F080E090E008958C
:1015A000869586958695E82FFF27E552FD4F808129
:1015B0009927277002C0959587952A95E2F79C0197
:1015C0002170307080FF03C081E090E00895C90170
:1015D000089508958091D802882359F48091D90202
:1015E000882339F48091DA02882319F481E090E0AD
:1015F000089580E090E008950895FF920F931F935F
:10160000CF93DF93FF2400E010E0C8E2D1E08881AF
:101610000E948A0A882311F0C80109C0F394219618
:101620000F5F1F4F8CE08F1594F78FEF9FEFDF91C7
:10163000CF911F910F91FF900895CF93C0E0EC2FB1
:10164000FF27E05EFE4F80810E948A0AEC2FEF5F49
:10165000882319F08E2F992705C0CE2FE83078F314
:1016600080E090E0CF910895CF93C0E0EC2FFF276A
:10167000E05EFE4F80810E94AA0AEC2FEF5F882374
:1016800019F08E2F992705C0CE2FE83078F380E02F
:1016900090E0CF91089580918F0210928F02992748
:1016A0000895282F883290F4869586958695E82FA0
:1016B000FF27EB56FD4F277081E090E002C0880FB6
:1016C000991F2A95E2F72081282B208308950895F9
:1016D000282F883290F4869586958695E82FFF27E7
:1016E000E057FD4F277081E090E002C0880F991FFE
:1016F0002A95E2F72081282B208308950895282F2A
:101700008832A0F4869586958695E82FFF27E057C6
:10171000FD4F277081E090E002C0880F991F2A9545
:10172000E2F7982F9095808189238083089508950A
:10173000282F883218F080E090E0089586958695ED
:101740008695E82FFF27E057FD4F277081E090E056
:1017500002C0880F991F2A95E2F720812823822F43
:10176000992708950895282F8832A0F486958695A4
:101770008695E82FFF27EB56FD4F277081E090E01C
:1017800002C0880F991F2A95E2F7982F90958081C3
:101790008923808308950895282F869586958695B8
:1017A000E5E9F2E0E80FF11D80819927277002C07A
:1017B000959587952A95E2F781709070089510921B
:1017C000990210929802109297021092960210922B
:1017D000950210929402109293021092920210922B
:1017E00091021092900208950F931F93CF9302E6F7
:1017F00011E0CFE0F80181918F010E94B30BC1503D
:10180000C7FFF8CFCF911F910F910895803138F421
:10181000E82FFF27EE59FE4F80810E94510B08955B
:101820000895803138F4E82FFF27EE59FE4F80816C
:101830000E94680B08950895803118F020E030E090
:1018400009C0E82FFF27EE59FE4F80810E94CC0B84
:10185000282F3327C9010895803118F080E090E0E7
:101860000895E82FFF27EE59FE4F80810E94980BC4
:10187000992708950895883138F4E82FFF27E65B0B
:10188000FE4F80810E94510B08950895883138F4ED
:10189000E82FFF27E65BFE4F80810E94680B0895CA
:1018A0000895883138F4E82FFF27E65BFE4F8081EA
:1018B0000E94B30B089508950F931F93CF930AE4EA
:1018C00011E0C7E1F80181918F010E94B30BC15073
:1018D000C7FFF8CFCF911F910F910895E82F815046
:1018E000883030F4FF27EF5BFE4F80810E94510B60
:1018F000089508951F93CF93182F81E0E82FFF27B5
:10190000C82FCF5F811731F4EF5BFE4F80810E94BB
:10191000510B05C0EF5BFE4F80810E94B30B8C2FF3
:10192000C93060F3CF911F910895E82F815088301E
:1019300030F4FF27EF5BFE4F80810E94B30B0895C8
:101940000895E82F8150883030F4FF27EF5BFE4F79
:1019500080810E94680B08950895E82F8150883097
:1019600040F4FF27EF5BFE4F80810E94980B992780
:10197000089580E090E008950895E82F8150883020
:1019800048F4FF27EF5BFE4F80810E94CC0B282F8D
:10199000332702C020E030E0C90108950F931F9360
:1019A000CF9302E411E0C7E0F80181918F010E941A
:1019B000B30BC150C7FFF8CFCF911F910F9108957E
:1019C0008D3038F4E82FFF27EB5CFE4F80810E94BA
:1019D000510B089508958D3038F4E82FFF27EB5C04
:1019E000FE4F80810E94680B08950895E5E3F1E0C1
:1019F000E80FF11D80810E94980B992708950F939D
:101A00001F93CF9305E311E0CCE0F80181918F01A2
:101A10000E94B30BC150C7FFF8CFCF911F910F9118
:101A200008950E94FF0C84E00E94B30B83E00E94A3
:101A3000B30B88E00E94B30B81E00E94B30B82E0FD
:101A40000E94B30B0895CF93C82F84E00E94B30B7C
:101A5000C23021F483E00E94680B0FC083E00E9433
:101A6000B30B83E00E947F0BC13011F483E003C00D
:101A7000CF3F19F484E00E94510BCF910895CF938A
:101A8000C82F0E94110DC7FF03C086E10E943B0CC6
:101A90008C2F829586958695837080FF03C085E1A3
:101AA0000E943B0CCF7311F48C2F15C0C73110F47A
:101AB0008FEF11C0C43218F4CC5080E00CC0C0339A
:101AC00018F4C85181E007C0CC3318F4C45282E046
:101AD00002C083E0C0530E94230DCC2321F484E193
:101AE0000E943B0C07C0EC2FFF27E65DFE4F808174
:101AF0000E94510BCF910895F894DF98E5E9F2E048
:101B000080818FB9779BFECF319682E0E939F80763
:101B1000B9F3B4F3DF9A78940895A0E9B2E0E5E967
:101B2000F2E024E080819D91892B8193215027FF51
:101B3000F9CF0895A0E9B2E0E5E9F2E024E09D9153
:101B40009095808189238193215027FFF8CF0895B4
:101B5000A0E9B2E0E5E9F2E034E020819C91822F37
:101B6000892319F09095292320831D9231503196B5
:101B700037FFF3CF0895AC0120E0322F61157105D6
:101B800081F0FA01E30FF11D80812827E22FFF2762
:101B9000EE58FE4F20813F5F832F992786179707C6
:101BA00080F3822F992708950F931F93CF93DF938C
:101BB0006115710549F08C01EB01F80181918F01EC
:101BC0000E9492062197C9F7DF91CF911F910F9143
:101BD00008950F931F939C0102EE12E082E480931C
:101BE000E2021092E30282E08093E402832F9927BD
:101BF0008093E5022093E60265E070E0C8010E9450
:101C0000BB0D8093E70266E070E0C8010E94D40D2E
:101C10001F910F9108950F931F9302EE12E090E829
:101C20009093E2021092E30291E09093E402809399
:101C3000E50264E070E0C8010E94BB0D8093E602FB
:101C400065E070E0C8010E94D40D1F910F910895C6
:101C50001F920F920FB60F921124EF92FF921F93D3
:101C60002F933F934F935F936F937F938F939F93A4
:101C7000AF93BF93CF93DF93EF93FF9393B1809193
:101C80007202882309F4E4C080919B02803448F4F6
:101C9000E82FFF27EE5DFC4F90838F5F80939B02C0
:101CA00004C00E940B0E10929B0220919B022330D5
:101CB00008F4CEC0F090220380912303682F772789
:101CC000762F6627809124039927682B792B332759
:101CD000CB0104962817390708F4BAC0FB01EE5D62
:101CE000FC4F1381EB012396BE0182E293E00E9438
:101CF000BB0D181791F0BE0182E293E00E94BB0D6C
:101D000099270E94FA0610929B0280E00E940B0E17
:101D10000E94F40B0E947C0D9DC08F2D992781316C
:101D2000910551F18231910544F48130910509F416
:101D300088C0409709F460C086C08034910521F0C6
:101D40008134910541F07FC08091A8029091A90251
:101D50000E94E90D7BC080912403823009F073C09A
:101D6000809125039927982F882720912603820F99
:101D7000911D0E9417056AC080912403823009F0EA
:101D800062C08091250390912603C82FDD2763E070
:101D9000CC0FDD1F6A95E1F7C90FD11D89E1809352
:101DA000E2021092E30280E18093E4020F2EF5EE4E
:101DB000EF2EF2E0FF2EF02DC295D295D07FDC27DA
:101DC000C07FDC271FE0CE010E949A10F7018193AB
:101DD0007F011150219617FFF6CF63E170E082EE8C
:101DE00092E00E94BB0D8093F50264E170E082EE08
:101DF00092E00E94D40D2AC080912403823119F50B
:101E00008091250390912603C82FDD2733E0CC0F66
:101E1000DD1F3A95E1F7C90FD11D27E2E22E23E03D
:101E2000F22E94E0CC0FDD1F9A95E1F71FE0BE0182
:101E3000F70181917F010E945B101150219617FFDD
:101E4000F6CF81E001C080E00E940B0E10929B0251
:101E50000E94F40BFF91EF91DF91CF91BF91AF9171
:101E60009F918F917F916F915F914F913F912F91B2
:101E70001F91FF90EF900F900FBE0F901F9018953D
:101E80000E94B7098091D7028E30D1F30E94DF0BF8
:101E90000E947C0D089590E03A98803408F08FE31A
:101EA000611160E4442311F440E801C0492F882304
:101EB00049F0862B842B85BB3A9A9F5F9832E8F3D2
:101EC000399A0895642B65BB08950895882311F00D
:101ED000AE9A01C039983A9808957F928F929F9256
:101EE000AF92BF92CF92DF92EF92FF920F931F9328
:101EF000CF93DF93EE24FF248824982C0E94EE04D5
:101F00000E94F40B7090DE02670157010E94B7092E
:101F10008091D702843019F00E942908BEC08091B8
:101F2000B0020E941C0C882331F40E94F40B8091B3
:101F3000B0020E94060C0E944B0B882309F1472D2A
:101F400055278091DE02992701969C01207F3170F0
:101F5000821B930B2091B0024817590721F42223CA
:101F600039F0215003C02F3019F02F5F2093B002B9
:101F70006091B00284E090E00E940D057090DE0256
:101F80008E2D0E94230D992019F081E00E94510BA3
:101F9000882019F082E00E94510B00E0C3E7D2E0F4
:101FA00088810E94AA0A8823B9F0102F1A0D195EA1
:101FB000492D682D812F0E944B0F892D992756E0BE
:101FC000880F991F5A95E1F7812B0E94CD08812F28
:101FD0000E943F0D41E0842E88810E94CA0A882316
:101FE00079F0202F2C0D295E892D992736E0880F56
:101FF000991F3A95E1F7822B0E94F1080E94110D7A
:102000000F5F21960D3060F28FE00E94AA0A8823AC
:1020100051F082E0E816F104D4F40894E11CF11CBC
:102020008CE090E010C08EE00E94AA0A882379F02C
:102030009FEFE9169FEFF90651F04CF00894E10884
:10204000F10884EF9FEFA80EB91EC80ED91E85E1D6
:102050000E94AA0A882371F080E0992009F481E0A7
:10206000982E882321F081E00E94510B03C081E06B
:102070000E94B30B83B399278F739070892B09F457
:1020800045CF0E94EA0A882309F440CF80E00E94ED
:10209000660F0E94110D882439CFDF91CF911F91D7
:1020A0000F91FF90EF90DF90CF90BF90AF909F90F7
:1020B0008F907F900895282FF89495E0C0980000A5
:1020C0000000000000009FB9779BFECF00000000D9
:1020D000000000001FB8779BFECF8FB1C09A0000B0
:1020E00000000000000080FDE9CFC0980000000063
:1020F00086E08FB9779BFECF00000000C09A0000F9
:10210000000000000000C0980000000082E08FB9CD
:10211000779BFECF872F99278FB9779BFECF6FB91B
:10212000779BFECF2FB9779BFECF00000000C09AAF
:10213000789408959C01F894C0980000000083E012
:102140008FB9779BFECF832F99278FB9779BFECFCF
:102150002FB9779BFECF000000001FB8779BFECF02
:102160008FB1C09A7894992708951092860310929F
:102170008D031092820380E00E94660F0E94DF0BA5
:102180000E94A80D0E944B0B08951092870384E2D1
:102190000E94B30B0E94DF0B0E94A80D10928D03CA
:1021A00080E00E94660F089581E08093870384E2B7
:1021B0000E94510B0E94F40B0895892F9927282F14
:1021C0002F71822F992787FD909534E096958795FA
:1021D0003A95E1F7892B09F0206E822F992787FD28
:1021E00090950895209184032770809184039091A5
:1021F0008503F3E096958795FA95E1F7622F8F7046
:102200000E94391560918403709185039B014427D6
:102210005527DA01C90180709078A070B070892FBD
:102220009A2FAB2FBB278093A202DA01C9018070DD
:102230009074A070B070892F9A2FAB2FBB2780931A
:10224000A4022070307240705070BB27A52F942FCD
:10225000832F8093A30210928A03CB010E94DD108A
:102260009927089581E08093860381E20E94510BB3
:102270001092A4028091A4028093A3028091A302F1
:102280008093A2021092820310928D0380916203C8
:102290009091630390938503809384038F5F9F4F96
:1022A00089F01092890310928A031092A7020E946B
:1022B000F21080939D028091810280FDFCCF81E02D
:1022C000809382030E94F40B089580919D028823DD
:1022D00021F483E00E94B30B0CC087FF07C083E0AA
:1022E0000E94B30B84E00E94510B089583E00E948A
:1022F000510B84E00E94B30B08950895FF920F9351
:102300001F93CF93DF93C82FDD2703E0CC0FDD1F92
:102310000A95E1F7C60FD11D15E0CC0FDD1F1A9508
:10232000E1F7BFE0FB2EC050D84F02E613E0CE012C
:102330000E949A109927982F8827F801808391830B
:10234000CE0101960E949A10282F3327F801808130
:102350009181822B932B819391938F01FA942296F2
:10236000F7FEE5CFDF91CF911F910F91FF90089578
:10237000FF920F931F93CF93DF93C82FDD2753E076
:10238000CC0FDD1F5A95E1F7C60FD11D45E0CC0FEC
:10239000DD1F4A95E1F73FE0F32E02E613E0C0505F
:1023A000D84FF80180819181892F9927BE010E9421
:1023B0005B102196F801819191918F01BE010E94DD
:1023C0005B10FA942196F7FEECCFDF91CF911F912D
:1023D0000F91FF9008951F93CF93DF930E94EE0417
:1023E0008091DE028770809383031092880310929D
:1023F0008703109286031092820310928D0310922D
:1024000089038FEF9FEF909385038093840310924D
:1024100082020E94F40B0E94A80D0E94B7098091CD
:10242000D702813071F00E94F40410928D03109253
:10243000820380E00E94660F0E94DF0B0E947C0DE9
:10244000EEC280918703882361F5809186038823FB
:1024500041F50E944B0B882359F08091DE02877072
:1024600080938303609188030E947E110E94F40B85
:10247000809183030E94060C0E941D0BC82F8823A5
:1024800059F00E94FF0C8C2F815080938803682F95
:10249000809183030E947E11809188038F5F0E9448
:1024A0006E0C81E00E94AA0A882379F0809186034D
:1024B000882319F00E94B51008C0809187038823F3
:1024C00011F00E94C5100E9432118091860388236A
:1024D00029F480918703882309F463C080918903DC
:1024E0000E942C0C882311F40E94A80D809189036E
:1024F0000E94110C80918403909185038F5F9F4F00
:1025000021F40E94110D80E046C080E00E94B30BD0
:10251000809184039091850343E0969587954A9531
:10252000E1F78F700E94060C8091840390918503DF
:1025300097FF04C088E00E94510B03C088E00E940E
:10254000B30B8091840390918503AA27BB273EE0BB
:10255000B695A795979587953A95D1F78170907024
:10256000892B21F081E00E94510B03C081E00E9481
:10257000B30B8091840390918503AA27BB272DE09C
:10258000B695A795979587952A95D1F78170907004
:10259000892B21F082E00E94510B03C082E00E944F
:1025A000B30B88E00E94AA0A882331F483E00E94DA
:1025B000AA0A882309F478C010918603112309F030
:1025C00073C0812F0E94660FC0918703CC2309F44A
:1025D00042C088E00E94AA0A8823D1F08091890332
:1025E0009927019640976CF480918903E82FFF2783
:1025F000EE0FFF1FEE59FC4F808191818F5F9F4F3F
:1026000019F41093890330C0809189038F5F20C033
:10261000809189038823C9F48091890399270196C1
:10262000409714F580918903E82FFF27EE0FFF1FD5
:10263000EE59FC4F808191818F5F9F4FA9F080916F
:1026400089038F5F80938903E7CF8091890381504D
:102650008093890309C088E00E94AA0A882321F098
:102660000E94D410C093890380918903E82FFF272B
:10267000EE0FFF1FEE59FC4F8081918190938503EF
:102680008093840310928D038F5F9F4F69F00E94A7
:10269000F21080939D0210928A038091810280FD46
:1026A000FCCF81E080938D0387E10E94AA0A8823F2
:1026B00039F1809187038823E9F080918903992774
:1026C0000196409764F480918903E82FFF27EE0F6D
:1026D000FF1FEE59FC4F8FEF9FEF828393838FEFA5
:1026E0009FEF90938503809384030E94C51080E040
:1026F0000E94B30B60918803809183030E94B811FC
:1027000080918703882309F47CC180918403909190
:1027100085038F5F9F4F09F40FC184E10E94AA0ACD
:10272000882311F180918903E82FFF27EE0FFF1F07
:10273000EE59FC4F8081918120E030E88227932779
:10274000808391838081918190938503809384031A
:10275000AA27BB2780709078A070B070892F9A2F1D
:10276000AB2FBB278093A20285E10E94AA0A88238F
:1027700011F180918903E82FFF27EE0FFF1FEE591B
:10278000FC4F8081918120E030E482279327808371
:102790009183808191819093850380938403AA27FC
:1027A000BB2780709074A070B070892F9A2FAB2FC8
:1027B000BB278093A40286E10E94AA0A882311F114
:1027C00080918903E82FFF27EE0FFF1FEE59FC4F82
:1027D0008081918120E030E282279327808391835A
:1027E000808191819093850380938403AA27BB27DE
:1027F00080709072A070B070892F9A2FAB2FBB277A
:102800008093A3028FE00E948A0A882331F48EE02D
:102810000E948A0A882309F47DC00E94FD0AC82FFD
:10282000DD27C7FDD0958FE00E94AA0A882329F4EE
:102830008EE00E94AA0A882351F00E94A80D0E94EF
:10284000FF0C83E00E94B30B84E00E94B30B8FE087
:102850000E948A0A882349F183E00E94510B8FEF7E
:10286000CF3FD807C9F00E94A80D20918403309172
:102870008503307E9C2F8827282B392B30938503A6
:102880002093840380918903E82FFF27EE0FFF1F19
:10289000EE59FC4F2083318380918403909185030E
:1028A0000E94DD1080939D0232C08EE00E948A0A51
:1028B000882309F441C084E00E94510B2FEFCF3FE1
:1028C000D207E1F00E94A80D209184033091850386
:1028D000307E2C97CF71D0709C2F8827282B392BD6
:1028E000309385032093840380918903E82FFF2789
:1028F000EE0FFF1FEE59FC4F20833183809184033C
:10290000909185030E94DD1080939D02845F0E9458
:10291000EB0C12C08FE00E94CA0A882329F48EE0D3
:102920000E94CA0A882341F083E00E94B30B84E02E
:102930000E94B30B0E94A80D8FE00E948A0A882390
:1029400009F05FC08EE00E948A0A882309F059C00E
:102950000E94340BC82F882329F40E944B0B882334
:1029600009F447C00E94CE0C0E94F40BCC2359F40A
:1029700080918403909185038F5F9F4F29F0C091D0
:102980008403C77001C0C15010928D0380E00E9483
:10299000660F4091DE02242F332763E0220F331F9E
:1029A0006A95E1F78C2F9927282B392B30938503D3
:1029B0002093840380918903E82FFF27EE0FFF1FE8
:1029C000EE59FC4F208331836C2F842F0E943915E0
:1029D00010928A031092A3028091A3028093A40212
:1029E0008091A4028093A20210929D0281E08093C4
:1029F0008D030E9465118091840387708F5F0E9410
:102A00007A0C80918603882309F407CD0E94651112
:102A10008091840387708F5F0E947A0CFECCDF91D7
:102A2000CF911F91089510928A0381E080938B03C8
:102A300081E20E94510B80E00E94660F0E94EE042A
:102A40008091810280FDFCCF81E080938D03089509
:102A500081E08093870384E20E94510B0E94F40B73
:102A600080E00E94060C0E94F40480E00E94660F41
:102A70000895EF92FF920F931F93CF93DF93182F38
:102A8000062F0E947C0DC12FDD2723E0CC0FDD1F18
:102A90002A95E1F7C00FD11D94E0CC0FDD1F9A9568
:102AA000E1F780E9E82E83E0F82E1FE0CE010E94D6
:102AB0009A10F70181937F011150219617FFF6CFED
:102AC0000E947C0DDF91CF911F910F91FF90EF90AD
:102AD0000895EF92FF920F931F93CF93DF93182FD8
:102AE000062F0E947C0DC12FDD2753E0CC0FDD1F88
:102AF0005A95E1F7C00FD11D40E9E42E43E0F42ED2
:102B000034E0CC0FDD1F3A95E1F71FE0BE01F7017D
:102B100081917F010E945B101150219617FFF6CF23
:102B20000E947C0DDF91CF911F910F91FF90EF904C
:102B300008951092870384E20E94B30B0E945C0CFC
:102B40000E94F40B8091DE020E94060C0E94EE04AB
:102B500080E00E94660F08950E94F40410928D0395
:102B60000E945C0C0E94F40B8091DE020E94060C15
:102B700010928B0381E20E94B30B80E00E94660FEB
:102B8000089581E080938F030E94EE0480E00E940C
:102B9000660F0E945C0C80E00E94680B8091DE0250
:102BA0000E94060C80918C038F5F0E946E0C08952A
:102BB00010928F0380E00E947F0B0E945C0C0E94A9
:102BC000F40B0895EF92FF920F931F93CF93DF932F
:102BD00010928C031092870310928B0310928F0334
:102BE00010928D0310928A031092A7021092820213
:102BF0000E94B7098091DE0280938E0360918C035E
:102C00000E9439150E94DF0B8091DE020E94060CA3
:102C10000E94EE040E94B7098091D702833081F0B0
:102C20000E94F40410928D0380E00E94660F0E94BF
:102C30003A090E940B090E94DF0B0E947C0D8CC296
:102C400090918E038091DE029817F9F080918B03AA
:102C5000882311F00E94AC1580918703882311F01E
:102C60000E9499159091DE0290938E0380918F03BC
:102C7000882329F460918C03892F0E9439150E94C2
:102C8000F40B8091DE020E94060C80918B03882356
:102C9000F9F4809187038823D9F480918C038F5FA6
:102CA0000E946E0C0E941D0BC82F882389F00E9481
:102CB000FF0C8C2F0E946E0C6C2F615060938C0364
:102CC00080918F03882321F480918E030E9439150F
:102CD00080E00E94AA0A882399F080918B038823C0
:102CE00079F082E20E94510B00E913E0CFE00E94EC
:102CF0005500F80181938F01C150C7FFF8CF0CC078
:102D000080E00E94CA0A882339F080918B038823CF
:102D100019F082E20E94B30B81E00E94AA0A882384
:102D2000A9F080918F03882311F00E94D81580911B
:102D30008B03882319F00E94AC1508C0809187038B
:102D4000882311F00E9499150E94131580918B031E
:102D5000882329F480918703882309F427C10091EF
:102D60008A03E02EFF24E701C057DC4F18811F7350
:102D700085E10E94AA0A882331F01F3321F088815F
:102D800090E48927888386E10E94AA0A882349F073
:102D90001F3339F0F701E057FC4F808190E8892715
:102DA00080831F3341F0112331F0173110F4CFEF3E
:102DB0000DC0143210F4C0E009C0103310F4C1E0AB
:102DC00005C01C3310F4C2E001C0C3E084E10E94DE
:102DD000AA0A811110E08FE00E94AA0A882339F024
:102DE0001F3329F0112319F01C160CF0145F8EE02C
:102DF0000E94AA0A882341F01F3331F0112321F0E9
:102E0000CF3F11F00CF01C5084E00E94AA0A8823E6
:102E100031F08CE0C802C0011124182F195E89E03E
:102E20000E94AA0A882331F08CE0C802C001112454
:102E3000182F185E85E00E94AA0A882331F08CE0E2
:102E4000C802C0011124182F175E8AE00E94AA0A46
:102E5000882331F08CE0C802C0011124182F165EBF
:102E6000C3300CF063C086E00E94AA0A882331F0C8
:102E70008CE0C802C0011124182F155E87E00E9463
:102E8000AA0A882331F08CE0C802C0011124182F4F
:102E9000145E8BE00E94AA0A882331F08CE0C802FD
:102EA000C0011124182F135E81E10E94AA0A882311
:102EB00031F08CE0C802C0011124182F125E8CE0A2
:102EC0000E94AA0A882331F08CE0C802C0011124B4
:102ED000182F115E82E10E94AA0A882331F08CE04B
:102EE000C802C0011124182F105E8DE00E94AA0AAA
:102EF000882331F08CE0C802C0011124182F1F5D17
:102F000080E10E94AA0A882331F08CE0C802C00147
:102F10001124182F1E5D83E10E94AA0A882331F034
:102F20008CE0C802C0011124182F1D5D202F33270B
:102F3000F901E057FC4F80818F3F11F41F3319F4E2
:102F40008081807C182BE901C057DC4F88811817DD
:102F5000F9F080918703882331F080E00E94660FAA
:102F600081E00E942907188380918703882381F0DC
:102F7000812F82958695869583708170912F991FF8
:102F80009927991F482F692F812F8F730E944B0F0C
:102F90001F3F39F0812F0E943F0D80E00E94B30B4C
:102FA00005C00E94110D80E00E94510B88E00E9434
:102FB000AA0A882331F483E00E94AA0A882309F42C
:102FC0009BC080918703882309F46AC080E00E9437
:102FD000660F81E00E94290788E00E94AA0A8823E0
:102FE000B1F080918A039927019640974CF4809123
:102FF0008A03E82FFF27E057FC4F80818F3F19F4A9
:1030000010928A0320C080918A038F5F1AC080913A
:103010008A03882399F480918A038F30A0F48091E9
:103020008A03E82FFF27E057FC4F80818F3F59F03C
:1030300080918A038F5F80938A03EDCF80918A030A
:10304000815080938A030E94F40B80918A030E942E
:10305000060C80918A03E82FFF27E057FC4F808100
:103060008093A7028F3F51F481E00E94B30B82E06E
:103070000E94B30B80E00E94510B3EC080E00E9492
:10308000B30B8091A702982F929596959695937081
:103090009170282F221F2227221F492F622F25C01F
:1030A00088E00E94AA0A882339F1C0918B03CC23BF
:1030B00019F50E942815C0938A0380918A03E82F8E
:1030C000FF27E057FC4FE081E093A702EF3FA1F01C
:1030D0008E2F829586958695837081709E2F991F7D
:1030E0009927991F482F692F8E2F8F730E944B0F9E
:1030F0008091A7020E943F0D87E10E94AA0A8823BF
:1031000009F488CD80918703882381F080918A0318
:1031100099270196409744F480918A03E82FFF276E
:10312000E057FC4F8FEF81830E94991580918B03AC
:10313000882311F00E94AC1580918F03882349F0F9
:1031400060918C038091DE020E9469150E94D8155F
:1031500061CD0E94C1155ECDDF91CF911F910F917E
:10316000FF90EF90089540E0DB01FC0190818C918D
:10317000981719F080E090E0089580818F3F19F44E
:1031800081E090E008954F5F31961196403270F3E0
:1031900081E090E008950895EF92FF920F931F93BE
:1031A000CF93FF24E090D70280918202882319F404
:1031B0000E94EE040BC00E94F404809182028130D0
:1031C00019F40E94720902C00E946B090E94DF0B71
:1031D0000E94A80D1092C0038091C0038093A003A9
:1031E0008FEF8093C1038091C1038093A10381E09D
:1031F0000E946E0C1092E1031092890310928A03D0
:1032000010928503109284031092E00310929C02A6
:1032100010929D020E94F40B8091D7028F3021F012
:103220008B3011F08730D1F48091DE021AC01092F9
:10323000E1030E943A090E940B0910929C0210922D
:103240009D021092A3021092A2021092A4020E9468
:10325000DF0B0E94A80D0E947C0DFEC28091DE0251
:1032600087708093A1028093A0028091DE020E9469
:10327000060C0E94B7098091D7028E15C1F687E12E
:103280000E94AA0A882329F180919E0290919F02B0
:1032900086509D40D0F480919E0290919F028E5462
:1032A000914098F020919E0230919F0280E69AEE24
:1032B000B9010E94321C70939F0260939E0280911C
:1032C0009E0290919F020E94170510929F021092F9
:1032D0009E0280E00E94AA0A882349F00E94FF0C07
:1032E0000E94A80D82E20E94510B1092A50280E07C
:1032F0000E94CA0A882329F1A2EEB3E0E0EAF3E0D3
:10330000CFE18D918193C150C7FFFBCF8091E10345
:103310008823A1F4A0EAB3E0E0ECF3E0CFE18D91E3
:103320008193C150C7FFFBCF80919C0280939D0287
:1033300083E00E94B30B84E00E94B30B82E20E9400
:10334000B30B80E00E948A0A882361F1C0E080917B
:10335000A502C81760F4EC2FFF27EE51FC4F8081C7
:10336000883028F48F5F0E946E0CCF5FF0CF0E94F0
:10337000340BC82F882309F44EC18091A5028032F6
:1033800008F049C1E82FFF27EE51FC4FC150C08320
:103390008F5F8093A502E82FFF27EE51FC4F8FEF40
:1033A000808339C18FE00E948A0A882331F48EE03D
:1033B0000E948A0A882309F46DC00E94FD0AC82F62
:1033C0008FE00E94AA0A882329F48EE00E94AA0AAC
:1033D000882339F00E94FF0C0E94A80D82E20E940F
:1033E000B30B8FE00E948A0A882301F184E00E94D7
:1033F000B30B83E00E94510BCF3F11F0C0939C02AE
:1034000080919D0287FD0AC00E94F60C882331F44A
:103410000E94A80D80919D020E94EB0C90919C024D
:1034200080919D02981761F1892F28C08EE00E943B
:103430008A0A882329F183E00E94B30B84E00E946A
:10344000510BCF3F19F0CC50C0939C0280919D024C
:10345000181664F0845F0E94F60C882339F40E94E9
:10346000A80D80919D02845F0E94EB0C90919C02BC
:1034700080919D02981721F0892F845F0E94E00CB3
:103480008091E103882309F0C6C080919C0280935B
:103490009D02C1C08FE00E94CA0A882329F48EE0F1
:1034A0000E94CA0A882321F00E94FF0C0E94A80DE6
:1034B0000E941D0BC82F882331F40E944B0B8823D8
:1034C00009F446C01FC00E94CE0CC150C093A00397
:1034D0008091A0038093E2038FEF8093A1038091FA
:1034E000A1038093E3038091E103882319F5A0EA07
:1034F000B3E0E0ECF3E0CFE18D918193C150C7FFE1
:10350000FBCF18C08091D7028F3021F08B3011F0A3
:10351000873019F48091DE0203C08091DE0287704B
:103520008093A0028091E103882321F48091A0027E
:103530008093A1028091E103882351F40E94F40B4F
:103540008091A0020E94060C80919C0280939D02B3
:1035500060EC73E080EA93E00E94B3188823F9F4EA
:103560008091A1038F3F49F48091C1038F3F29F4DB
:103570008091C0038F5F0E94A10CC0E000EA13E0BD
:10358000F8018081893008F044C0D8018D918D0107
:103590008F5F0E946E0CCF5FC03290F33AC0C0E0E4
:1035A00000EC13E0F8018081893098F58091E10307
:1035B0008823E1F08091E003E82FFF27E054FC4FDF
:1035C000D8019C918081981789F48C918F5F0E941B
:1035D000AD0C8823C9F4F80180818F5F0E94950C9F
:1035E000D8018C918F5F0E94A10C0EC0F8018081E0
:1035F0008F5F0E94AD0C882311F00E94A80DD801A6
:103600008C918F5F0E946E0CCF5F0F5F1F4FC03297
:1036100048F20E9465118091E103882351F1809165
:103620008202823089F4809183029091840218167C
:103630001906FCF480918302909184020397909381
:1036400084028093830212C0813099F480918C02AD
:1036500090918D021816190664F480918C02909155
:103660008D02039790938D0280938C020E947400C8
:1036700000CE80918202823019F40E94C307F82E96
:1036800080918202882349F481E00E94AA0A88235B
:1036900021F08091E103882371F4809182028230CD
:1036A00021F4BCEFFB1639F02BC0813049F50E94A4
:1036B0005609882329F11092E10380E00E94660FE9
:1036C0000E940B0980918202813011F00E943A0918
:1036D00081E20E94B30B0E94A80D0E94F40B80911E
:1036E000D7028F3021F08B3011F0873019F48091A0
:1036F000DE0203C08091DE0287700E94060C68C063
:1037000080918202882349F481E00E94AA0A8823DA
:1037100021F08091E103882389F080918202823038
:1037200029F48F2D8A5F823048F052C0813009F031
:103730004FC00E944109882309F44AC081E20E94D7
:10374000510B8091D7028F3021F08B3011F08730F0
:1037500039F46091C0038091DE020E94391511C0D6
:103760008091DE026091C00387700E947E1180917B
:1037700062039091630390938503809384030E9476
:10378000F2101092A70280918202823019F4EBEFBE
:10379000FE1631F01092E00310928A031092890312
:1037A00010928102109284021092830210928D0274
:1037B00010928D0210928C0281E08093E1038AEFD7
:1037C0000E94230880918202813011F00E94160924
:1037D00086E10E94AA0A882389F090E08091A302E2
:1037E000882309F491E09093A302992321F082E0C9
:1037F0000E94510B03C082E00E94B30B85E10E943E
:10380000AA0A882389F090E08091A402882309F411
:1038100091E09093A402992321F081E00E94510B42
:1038200003C081E00E94B30B84E10E94AA0A8823AE
:1038300009F41FCD90E08091A202882309F491E061
:103840009093A202992321F088E00E94510B11CDA0
:1038500088E00E94B30B0DCDCF911F910F91FF9087
:10386000EF900895AA1BBB1B51E107C0AA1FBB1F05
:10387000A617B70710F0A61BB70B881F991F5A95FC
:10388000A9F780959095BC01CD010895A1E21A2E6B
:10389000AA1BBB1BFD010DC0AA1FBB1FEE1FFF1FF4
:1038A000A217B307E407F50720F0A21BB30BE40B44
:1038B000F50B661F771F881F991F1A9469F760958B
:1038C0007095809590959B01AC01BD01CF01089545
:1038D00064207F526563656976656420556E6B6E02
:1038E0006F776E204D4944493A203078000A0D0028
:1038F00004050607111210130409050A06070B1127
:103900000C120D1013201B191C1A180F0C0E0B0D86
:103910000A0920191A180C0B0A092221252320193B
:103920001A18241B1C0F0E0D04030A0C0B090801A6
:10393000020026271D1E1F1012111314151617053D
:10394000060700070E091C1B1215383F36312423C9
:103950002A2D70777E796C6B6265484F46415453CF
:103960005A5DE0E7EEE9FCFBF2F5D8DFD6D1C4C33F
:10397000CACD90979E998C8B8285A8AFA6A1B4B32F
:10398000BABDC7C0C9CEDBDCD5D2FFF8F1F6E3E49F
:10399000EDEAB7B0B9BEABACA5A28F88818693948F
:1039A0009D9A2720292E3B3C35321F1811160304FF
:1039B0000D0A5750595E4B4C45426F6861667374EF
:1039C0007D7A898E878095929B9CB1B6BFB8ADAA4F
:1039D000A3A4F9FEF7F0E5E2EBECC1C6CFC8DDDA4F
:1039E000D3D4696E676075727B7C51565F584D4ABF
:1039F0004344191E171005020B0C21262F283D3AAF
:103A000033344E49404752555C5B7671787F6A6D1E
:103A100064633E39303722252C2B0601080F1A1D0E
:103A20001413AEA9A0A7B2B5BCBB9691989F8A8D7E
:103A30008483DED9D0D7C2C5CCCBE6E1E8EFFAFD6E
:103A4000F4F3010409050A06070B110C120D1013FB
:00000001FF
